:0200000480007A
:100000006F008004732F2034930F80006308FF0378
:10001000930F90006304FF03930FB0006300FF038E
:10002000130F000063040F0067000F00732F2034CC
:1000300063540F006F00400093E19153171F0000BD
:1000400023223FFC6FF09FFF93000000130100008C
:10005000930100001302000093020000130300004C
:100060009303000013040000930400001305000034
:10007000930500001306000093060000130700001C
:100080009307000013080000930800001309000004
:1000900093090000130A0000930A0000130B0000EC
:1000A000930B0000130C0000930C0000130D0000D4
:1000B000930D0000130E0000930E0000130F0000BC
:1000C000930F0000732540F16310050097020000B4
:1000D000938202017390523073500018970200000F
:1000E00093824202739052309B021000939252030B
:1000F0009382F2FF7390023B9302F0017390023AF5
:100100007350403097020000938242017390523046
:10011000735020307350303093010000970200007C
:10012000938282EE73905230130510001315F5017F
:10013000635C05000F00F00F930110009308D005D9
:10014000130500007300000093020000638A0200A0
:1001500073905210B7B200009B82921073902230BD
:100160007350003097020000938242017390123462
:10017000732540F173002030B700008013D70000D2
:10018000B7030080930120006316772EB70000802C
:1001900013D710009B031000939313029383F3FF74
:1001A0009393E301930130006316772CB70000802E
:1001B00013D770009B031000939313029383F3FFF4
:1001C00093938301930140006316772AB700008060
:1001D00013D7E0009B031000939313029383F3FF64
:1001E000939313019301500063167728B7000080A2
:1001F0009B80100013D7F0019B0310009393130210
:100200009383F3FF93016000631677269300F0FF5A
:1002100013D700009303F0FF93017000631C772451
:100220009300F0FF13D710009B03F0FF9393F303A9
:100230009383F3FF93018000631E77229300F0FF06
:1002400013D770009B031000939393039383F3FFE2
:1002500093019000631077229300F0FF13D7E00022
:100260009B031000939323039383F3FF9301A00058
:10027000631277209300F0FF13D7F0019B03100067
:10028000939313029383F3FF9301B0006314771EDB
:10029000B72021219B80101213D70000B723212102
:1002A0009B8313129301C0006316771CB720212192
:1002B0009B80101213D71000B79390109B830309F3
:1002C0009301D0006318771AB72021219B80101268
:1002D00013D77000B74342009B8323249301E000AF
:1002E000631A7718B72021219B80101213D7E000E2
:1002F000B78300009B8343489301F000631C77168B
:10030000B72021219B80101213D7F0019303000026
:1003100093010001631077169B0010009390F00189
:1003200093D07000B703000193011001639470141F
:10033000130200009B0010009390F00113D770008F
:10034000130307001302120093022000E31452FE6D
:10035000B703000193012001631E73101302000014
:100360009B0010009390F00113D7E00013000000F1
:10037000130307001302120093022000E31252FE3F
:10038000B7030200930130016316730E13020000DD
:100390009B0010009390F0019380100013D7F001A0
:1003A00013000000130000001303070013021200E3
:1003B00093022000E31E52FC9303100093014001BE
:1003C000631A730A130200009B0010009390F0015F
:1003D00013D770001302120093022000E31652FE9E
:1003E000B703000193015001631677081302000060
:1003F0009B0010009390F0011300000013D7E00061
:100400001302120093022000E31452FEB70302000D
:100410009301600163107706130200009B00100037
:100420009390F0019380100013000000130000006F
:1004300013D7F0011302120093022000E31052FEC2
:1004400093031000930170016316770293504000EC
:100450009303000093018001639E700093001002DB
:1004600013D0A00093030000930190016314700067
:10047000631030020F00F00F6380010093911100B0
:1004800093E111009308D00513850100730000006B
:100490000F00F00F930110009308D0051305000022
:1004A00073000000731000C0000000000000000096
:0C04B00000000000000000000000000040
:1010000000000000000000000000000000000000E0
:1010100000000000000000000000000000000000D0
:1010200000000000000000000000000000000000C0
:1010300000000000000000000000000000000000B0
:081040000000000000000000A8
:040000058000000077
:00000001FF
